:04000000B6017228AB
:100008000800B616B61EB61236190F28FE39B70004
:10001800361503106D28361A1728A60036162E2016
:1000280003181C282608352003181C28B61E6D281E
:1000380027204C2036113612B6113A0884003808A9
:10004800841780042D283A0884003809800584170D
:100058008005080021204C20272048203708B619A1
:100068000138A2000830A300A20D03182120031CA8
:1000780027204C204820A30B382821204C203A0860
:10008800840038080005FF3E3B08840039092A2807
:100098003B08840039082428A301A200FF30A207E6
:1000A800031CA307031C6D280330A100E7305E2062
:1000B8005228A101FC3EA000A109031C6928FF30B9
:1000C8000000A00703186428A0076400A10F632894
:1000D8000800831303138312640008008316073093
:1000E8009F008312BE01BC01BD01BF016400F03056
:1000F8003F028A110A120318102A3F08EF3C8A119E
:100108000A12031CF1298A110A128E20BE008A11D4
:0C0118000A12F12901308A003F0800297A
:100200008207003400344F340034003400340734A3
:1002100000340734003414347F3414347F341434FD
:1002200024342A347F342A341234233413340834E7
:100230006434623436344934553422345034003412
:1002400005340334003400341C3422344134003487
:10025000003400340034413422341C341434083463
:100260003E3408341434083408343E340834083436
:100270000034503430340034003408340834083446
:1002800008340834003460346034003400342034DE
:1002900010340834043402343E3451344934453483
:1002A0003E34003442347F344034003442346134CC
:1002B0005134493446342134413445344B3431349B
:1002C0001834143412347F34103427344534453410
:1002D000453439343C344A344934493430340134B7
:1002E00071340934053403343634493449344934DB
:1002F000363406344934493429341E340034363413
:10030000363400340034003456343634003400348B
:100310000834143422344134003414341434143482
:100320001434143400344134223414340834023484
:100330000134513409340634323449347934413487
:100340003E347E341134113411347E347F344934D8
:100350004934493436343E34413441344134223412
:100360007F344134413422341C347F34493449349D
:10037000493441347F3409340934093401343E347A
:100380004134493449347A347F34083408340834E9
:100390007F34003441347F344134003420344034DD
:1003A00041343F3401347F3408341434223441342E
:1003B0007F3440344034403440347F3402340C3491
:1003C00002347F347F340434083410347F343E34B4
:1003D0004134413441343E347F34093409340934E2
:1003E00006340730BA001030B8000730BB000830C0
:1003F000B900A0308A0107203D088A0107203C0887
:100400008A0107203E088A01052014308A01502005
:10041000BC0A0319BD0ABF0A8A110A12031D7A28F1
:10042000BF016400E6303F028A110A120318062C4D
:100430003F08E53C8A110A12031CE72B8A110A12B5
:100440002522BE008A110A12E72B03308A003F08DA
:02045000002B7F
:1006000082073E344134513421345E347F3409341E
:100610001934293446344634493449344934313460
:10062000013401347F34013401343F3440344034E8
:1006300040343F341F342034403420341F343F349E
:100640004034383440343F34633414340834143480
:100650006334073408347034083407346134513457
:100660004934453443347F34413441340034003418
:10067000023404340834103420340034003441345B
:1006800041347F34043402340134023404344034BD
:1006900040344034403440340034013402340434B3
:1006A0000034203454345434543478347F3448344F
:1006B00044344434383438344434443444342034B6
:1006C00038344434443448347F3438345434543423
:1006D0005434183408347E340934013402340C3470
:1006E0005234523452343E347F34083404340434A7
:1006F0007834003444347D344034003400342034C1
:10070000403444343D347F3410342834443400348D
:10071000003441347F34403400347C3404341834A1
:10072000043478347C340834043404347834383471
:1007300044344434443438347C341434143414345D
:10074000083408341434143418347C347C340834B9
:100750000434043408344834543454345434203485
:1007600004343F344434403420343C344034403446
:1007700020347C341C342034403420341C343C3449
:100780004034303440343C34443428341034283439
:1007900044340C345034503450343C344434643495
:1007A00054344C3444340834363441340034003446
:1007B000003400347F3400340034003400344134D9
:1007C0003634083400340834043408340434073030
:1007D000BA001030B8000730BB000830B900A030B4
:1007E0008A0107203D088A0107203C088A0107206A
:1007F0003E088A01052014308A015020BC0A0319E2
:10080000BD0ABF0A8A110A12031D112A63008A0158
:02081000062CB4
:02400E00753DFE
:00000001FF
